:060000000C942B000C948F
:1000060000000C9400000C9400000C9400000C946A
:1000160000000C9400000C9400000C9400000C945A
:1000260000000C9400000C9400000C9400000C944A
:1000360000000C9400000C9400000C9400000C943A
:1000460000000C9400000C9400000C9400000000CA
:10005600F894EE27ECBBF1E0FBBFEBBFE5BFF8E1A0
:10006600F1BDE1BD8DE0A2E0BB27ED938A95E9F7EE
:1000760080E094E0A0E6ED930197E9F7E4E5F0E08F
:1000860085919591009761F0A591B5910590159090
:10009600BF01F00105900D920197E1F7FB01F0CF4A
:1000A600EFE5EDBFE4E0EEBFC0E6D1E00C945B0007
:1000B600EFEFE7BBE0E0E8BB01E010E00A31E0E08B
:1000C6001E076CF421E030E02930E0E03E0724F41E
:1000D6001FD0220F331FF8CF0F5F1F4FEFCF01E066
:1000E60010E00A31E0E01E078CF428E030E0213011
:1000F600E0E03E0744F00CD0D901E2E0F0E00E94D7
:10010600B8009F01F4CF0F5F1F4FEBCFD5CFFFCFC6
:10011600F901E095F095E8BBE8ECF0E0FA93EA9394
:100126000C949500E991F991309639F088EE93E0B8
:100136000197F1F7A8953197C9F70895E095F095DD
:10014600319608950024112490E1AA0FBB1F001CCC
:10015600111C0E1A1F0A18F40E0E1F1E01C0A160F4
:100166009A9599F7FD01D001089504D0EBDF0EF4BE
:10017600E5DF0895E894F7FF02C0E0DF6894B7FF73
:1001860006C0A095B095119600F8039400FA08955C
:00000001FF
